:080000000C9497000C94000021
:100008000C9400000C9400000C9400000C94000068
:100018000C9400000C9400000C9400000C94000058
:100028000C9400000C9400000C9400000C94000048
:100038000C9400000C9400000C94CA000C9400006E
:100048000C94FE000C9400000C9400000C9400002A
:100058000C9400000C9400000C9400000C94000018
:100068000C9400000C9400000C9400000C94000008
:100078000C9443010C9400000C9400000C940000B4
:100088000C9400000500FA00FF00FF000200C80001
:10009800CF00D900DF00E200E900000000003F06C1
:1000A8005B4F666D7D077F6F004079547C5873778E
:1000B8005E000100FF00FF000C00010000000000CE
:1000C80043434153543A0041542B55434153543A06
:1000D800004A50414E3A004F4B0043444154413A84
:1000E800004552524F520000010004008C000100EC
:1000F80005008E0001009202900001009302920018
:1001080001008C0594000100530ABA000100570A47
:10011800BC000100580ABE000100590AC0000100D5
:100128005A0AC2000000F894EE27ECBBF1E0F5BFD4
:10013800E5BFE0936C00EBBFF8E1F1BDE1BD8DE0F8
:10014800A2E0BB27ED938A95E9F780E090E1A0E073
:10015800B1E0ED930197E9F7E0EFF0E08591959133
:10016800009761F0A591B59105901590BF01F00138
:1001780005900D920197E1F7FB01F0CFEFEFEDBF8E
:10018800E0E1EEBFC0E9D2E00C9433020A92AA93F0
:10019800BA93EA93FA93EFB7EA93E0E0E2BF4A949E
:1001A8005A94A0919002B09191020E943317D0F412
:1001B800E0919002F09191023197E0939002F093D0
:1001C8009102A0919002B09191020E94331731F4EC
:1001D800A0919302A03014F023FE01C003C0EFEFFA
:1001E800E0939302E991EFBFF991E991B991A9914F
:1001F800099018950E9419130BB11CB1E02FEC71EE
:10020800E1F4A0919F05B0E0A157BA4F1C93A091CB
:100218009F05AF5FA0939F05A03119F4E0E0E0933C
:100228009F05A091A105AF5FA093A105A03129F476
:10023800E0E0E093A105689430F80E942113189536
:100248000A93E091A105E030E1F3E091A005F0E028
:10025800E157FA4F0081A091A005AF5FA093A005D8
:10026800A03119F4E0E0E093A005F894E091A1052D
:10027800E150E093A1057894E02F099108950E9438
:10028800191300919B0010919C00E02FEC71E1F490
:10029800A091B205B0E0AE55BA4F1C93A091B2053B
:1002A800AF5FA093B205A03119F4E0E0E093B20586
:1002B800A091B405AF5FA093B405A03129F4E0E0A4
:1002C800E093B405689431F80E94211318950A93B5
:1002D800E091B405E030E1F3E091B305F0E0EE55CC
:1002E800FA4F0081A091B305AF5FA093B305A03189
:1002F80019F4E0E0E093B305F894E091B405E15017
:10030800E093B4057894E02F56C0E0919B00E0722A
:10031800E1F3E881E0939C00219608950A9300E0B8
:100328000831D0F40E942913EC56FD4FDF01E0E3B9
:100338000E943013FF93EF93E5E9F2E0AF91BF918C
:10034800FF93EF93E3E1F0E00E94C616AF91BF91EF
:100358000E9434130F5FE4CF00E0003160F5E02F16
:10036800F0E0FF93EF93EDE5F4E0AF91BF91FF93D9
:10037800EF93E3E1F0E00E94C616AF91BF910E94AF
:1003880034130E942913E45AFB4FDF01E0E00E9476
:100398003013FF93EF93EEE5F4E0AF91BF91FF9335
:1003A800EF93E3E1F0E00E94C616AF91BF910E947F
:1003B80034130F5FD2CF09910895E3E09E2E9D99E3
:1003C80093949E9B02C093949394809903C0E92DC3
:1003D800E4509E2EA0E0B0E00E941017AE2FE1E09E
:1003E800EA1720F4A0E0B0E00E942417A1E0B0E0F2
:1003F8000E940C17E038A5E2FA0781F0A1E0B0E00E
:100408000E940C17E030ABE4FA0741F0A1E0B0E03D
:100418000E940C17E030A6E9FA0709F406C0E0E0EC
:10042800FBE4A1E0B0E00E941C170895A1E0B0E051
:100438000E940C17E038A5E2FA0711F4E7E60CC0B1
:10044800E030ABE4FA0709F406C0E030A6E9FA07A1
:1004580011F4E9E101C0E3E3E09399000895E8ECC1
:10046800F0E0FA93EA930E94A116EFEFEBBBEABB28
:10047800E8BBE0EFE7BBEFE9E5BBE4BBE3EFE2BBDA
:10048800E8EFE1BBEFEFE3B9EEE7E2B9EFEFE093B6
:100498006200EFE0E0936100EFEFE0936500EFE1C9
:1004A800E0936400E0E0E0BFE5E0E3BFE0E0E2BF46
:1004B800E1BFEFBDEEBDEDBDECBDE7BDE6BDEBBDFB
:1004C800EABDE9BDE8BDE0937900E0937800E5BDB9
:1004D800E4BDE3BDE0938B00E0938A00E0938900DC
:1004E800E0938800E0938100E0938000E093870028
:1004F800E0938600E0938500E0938400E093830016
:10050800E0938200E0936A00EABFE9BFE1E0E7BF59
:10051800E0E0E0937D00EBB9E8E9EAB9E6E0E093D2
:100528009500E0E0E0939000E3E3E9B9E0E0E093D0
:100538009B00E8E9E0939A00E6E0E0939D00E0E0A4
:10054800E0939800E3E3E0939900E0E8E8B9E0E09D
:10055800E0BDE8E1E1BDE8E0E1BD7894E0EEE5BBAF
:10056800E3E0E0936500E2E0E0938C050E949201ED
:100578000E94E1010E941A020E94B30EA895E09120
:10058800B405E03051F00E946B01E0938E05A09114
:100598008C05A23011F4EA9368D1E091A105E0300E
:1005A800D9F00E942401E0938E05E0918C05E33098
:1005B80029F4E0918E05EA93C5D60EC0E23029F4FD
:1005C800E0918E05EA93CBD607C0E43029F4E09198
:1005D8008E05EA930E94CC1205D50E94E20A4420B7
:1005E80021F4EAEF4E2E0E94E811E5E0E51510F43B
:1005F8000C944C03EAEF5E2EC3948394E8E1CE1684
:1006080008F0CC24EC2DF0E0FF93EF93E5E9F2E05D
:10061800AF91BF91FF93EF93E3E1F0E00E94C6161C
:10062800AF91BF91AE0FBF1FAC91E0E0EA1780F524
:10063800EC2DF0E0FF93EF93E5E9F2E0AF91BF9185
:10064800FF93EF93E3E1F0E00E94C616AF91BF91EC
:10065800AE0FBF1FEC91E150EC93EC2DF0E0FF934F
:10066800EF93E5E9F2E0AF91BF91FF93EF93E3E1F8
:10067800F0E00E94C616AF91BF910E94391341F471
:10068800EC2D0E943E13EC56FD4FDF01E4E3EC93A2
:10069800E1E08E1610F40C94C90388247724EE2424
:1006A800E0E1EE1648F4EE2D0E943E130E9444133A
:1006B80008F47394E394F4CFA0919302AF3F21F42C
:1006C800A0919202AF3F09F05FC0E0E1BE1608F0CA
:1006D800BB24EB2D0E943E130E94441310F00C948F
:1006E800C703EB2DF0E0FF93EF93EDE5F4E0AF9156
:1006F800BF91FF93EF93E3E1F0E00E94C616AF913C
:10070800BF91AE0FBF1FAC91EB2DF0E0FF93EF93BD
:10071800EDE5F4E0AF91BF91FF93EF93E3E1F0E0F3
:100728000E94C616AF91BF91AE0FBF1FAC91AA3001
:1007380090F4EB2DF0E0FF93EF93EDE5F4E0AF914B
:10074800BF91FF93EF93E3E1F0E00E94C616AF91EB
:10075800BF910E944B13EB2DF0E0FF93EF93EDE573
:10076800F4E0AF91BF91FF93EF93E3E1F0E00E94D3
:10077800C616AF91BF91AE0FBF1FAC91E4E0EA1768
:1007880010F4B0929202B394A394A0918C05A43073
:1007980081F020FC0BC022FC09C023FC07C0A091FB
:1007A8009002B09191020E94331709F002C00E9492
:1007B800100FE4CEFFCFA881A23018F0ECE8EA17BA
:1007C80020F4E0E0E09344060CC0E881E09345069D
:1007D800E0934606E09347060E945113E0E0E09359
:1007E80042066EC0E0914506E150E0934506E030D0
:1007F800A1F40E945713E4E0EC93A0914206AC38B0
:1008080010F0E0E007C00E945713E881EC93E091F4
:100818004406EF5FE093440604C00E945713E88142
:10082800EC93A0914206AC3818F0E0E0E09344065F
:10083800E881A0914706EA0FE093470641C0A881E6
:10084800AD3021F0E0E0E09344060BC00E9457135E
:10085800E0E0EC93E0914706E03019F4E1E0EA9338
:1008680031D0E0E0E09344062BC0E0914406E0304C
:1008780031F4A881AA3511F40E94511321C0E13046
:1008880059F4E881E03021F4E0914406EF5F01C0BB
:10089800E0E0E093440614C0E23029F4E881EA93EA
:1008A8000E94DF030DC0E33029F4E881EA930E9437
:1008B800F60306C0E43021F4E881EA930E94230499
:1008C800219608950E94371750E00E9462132081F4
:1008D8000E946D1330810E946D134081EFEFE09309
:1008E8004209A0918C05A230A1F4E09143060E9430
:1008F8007713E0934209A0914209A03318F0E4E38A
:10090800EA1708F406C0E0914306EF5FE093430658
:1009180051E00E946D1300810E946D1310813335E0
:1009280021F4A42FA0539A1609F007C02A930A931A
:100938001A935A93EA85EA9386D2343519F4EE81EC
:10094800EA93F2D60E943E172796089524971A93A1
:100958000A9310E100E1083150F40E942913EC5683
:10096800FD4FE081E03309F018E10F5FF4CF0E94FA
:100978007C130E94801300E0011740F40E942913A1
:10098800EC56FD4F0E9484130F5FF6CF0E94881328
:100998000E947C130E948C13E72DF0E0FA93EA93EF
:1009A800FE0134960E9490130E940C0EEA81EA938D
:1009B800A5D2EB810E949513E7D2EE81E0938D05D5
:1009C80019810881279608950E9499130E949E1301
:1009D800E981E03009F09AD20E94A31315C12B9740
:1009E80081E0A0E0B0E0E2EAF0E00E9445170E9452
:1009F8003717A989E0E0EA1710F00C949A0541E04E
:100A0800E0914206E3505E2F0E946D1310810E9410
:100A1800A713EF930E94AC13AF91EA2329F00E9429
:100A2800B113AE0FBF1F1C93E52FA09143060E9480
:100A3800BC16EF93AE81E9E00E94BC16AF91EA23A1
:100A4800EF930E94A713AF91EA23EF930E94AC1390
:100A5800AF91EA23C9F60E94B1130E943413FE0134
:100A68003796FA93EA930E94E6122E2FA22FE0E11E
:100A78000E94C116EF93A22FE1E00E94BC16AF912D
:100A8800EA2B11F020E040E0E0E0E21770F430E0FB
:100A9800303158F4E32F0E943E130E94441318F497
:100AA8002150203011F03F5FF3CF0E9499130E942C
:100AB8009E13EA89E03009F029D20E947C13E2E50E
:100AC800EA931CD2A22FE0E00E94AD16EF93A42F68
:100AD800E1E00E94AD16AF91EA23C9F000E0EFE033
:100AE800E017A0F0E32FF0E0FF93EF93EFE5F4E0D9
:100AF800AF91BF91FF93EF93E3E1F0E00E94C61638
:100B0800AF91BF910E94B9130F5FE9CF09C000E010
:100B1800EFE0E01728F0E0E3EA93F0D10F5FF8CFB9
:100B28000E94881331D2E989E0938D050E943E170F
:100B3800639608951A930A9310E000E0003150F587
:100B48000E9429130E944413E0F4E02FF0E0FF9381
:100B5800EF93EFE5F4E0AF91BF91FF93EF93E3E1FB
:100B6800F0E00E94C616AF91BF91EA0FFB1FFA93FF
:100B7800EA93E3E1F8E00E94C3130E945616E030BE
:100B880009F006C011E00E9429130E94CA1302C08E
:100B98000F5FD4CF103059F500E0003140F50E94C6
:100BA8002913E45AFB4FE081E030F9F4E02FF0E03C
:100BB800FF93EF93EFE5F4E0AF91BF91FF93EF93CD
:100BC800E3E1F0E00E94C616AF91BF91EA0FFB1F68
:100BD800FA93EA93E3E1F8E00E94C3130E946816CF
:100BE8000E9429130E94CA1302C00F5FD6CFE8C122
:100BF8000E9499130E949E13E981E03009F086D182
:100C08000E94D0130E94A313229608950A93A091DC
:100C18004509A23011F421FC01C043C0D4D10E947F
:100C280099130E949E130E94D013EEE4EA9366D1B2
:100C3800ECE40E94D6130E94DB13EEE20E94D61366
:100C4800F0E0FF93EF93EEE5F4E0AF91BF91FF93EF
:100C5800EF93E3E1F0E00E94C616AF91BF91AE0FAB
:100C6800BF1FEC910E94DB13ECE2EA9347D100E04E
:100C7800EFE0E017A0F0E981F0E0FF93EF93EFE5F4
:100C8800F4E0AF91BF91FF93EF93E3E1F0E00E94AE
:100C9800C616AF91BF910E94B9130F5FE9CF0E94AA
:100CA800DF130881229608950E9499130E949E13CB
:100CB8002DD10E947C13EDE4EA9320D1E0918C05BC
:100CC800E05D0E9495130E94E61308950A930E941E
:100CD8006D130081013319F4E0E0E0938C0572C0D4
:100CE8000A930E946D130081003319F4E2E0E09347
:100CF8008C05013319F4E3E0E0938C0563C0289771
:100D08000A9300E00E94EC130E94BC16EF93A02FF8
:100D1800E5E00E94B216AF91EA2381F0E02F0F5F61
:100D2800F0E0DE011196EA0FFB1FFF93EF930E949C
:100D38006D13E081AF91BF91EC93E4CFE02F0F5F8B
:100D4800F0E0DE0111960E943413FE013196FA9309
:100D5800EA930E94E612A1E0B0E00E941C170E94EC
:100D68001A020881299608950A930E946D1300813A
:100D7800003311F4E0E001C0E1E0A0E0B0E00E943F
:100D880024170E9475101EC00A930E94EC13AE1718
:100D9800B8F40E946D1300810C3579F40E946D132C
:100DA800E081EA930E946D13E081EA93EDB7FEB704
:100DB800FA93EA930F9376D70F910A9390D2E5CFDF
:100DC800689420F8099108950E943A17EFE1EA9390
:100DD80085D00E9480130E949E1398D0E0917208DB
:100DE800A0917308EA1761F1E0917308EF5FE0934F
:100DF80073080E94F2130081A0917308A43618F0BA
:100E0800E0E0E0937308003218F0EDE7E017A8F48B
:100E1800ECE5EA9373D00A93EDB7FEB7FA93EA9339
:100E28001F93EDB7FEB7FA93EA932F931BD72F9131
:100E38001F911A9363D02A9301C00A935FD0CECF33
:100E48000E94E6139DC0E881E0934509AC81AF306C
:100E5800B1F4EB81E73499F4EA81E33529F40E948F
:100E6800F7130E94E8040BC0ED3419F40E945806E9
:100E780006C0E23521F40E94F7130E94F304AC8106
:100E8800A231F1F4EB81E73451F4EA81ED3419F43D
:100E98000E946A0603C0E13209F4FFCF11C0E332B1
:100EA80079F4EA81E13419F40E94740609C0E23445
:100EB80019F40E94830604C0E33411F40E94B806B2
:100EC800AC81AF3149F4E0914306E250E093430628
:100ED8000E94C8060E94E80625960895E0E00E9450
:100EE800FC13EAE50E9407140E940C14E0E00E943B
:100EF80007140E94FC13E881EC932FC2E091D506F9
:100F0800EF5F0E940C14E881EC9327C20E943A1705
:100F1800A0914209AF3FA1F1E0914209E1701E2F73
:100F2800E0914209E695E1702E2FE0914309E2171E
:100F380019F4EF5FE0934309E0914409E11719F0D0
:100F4800EF5FE0934409E0914309E170E0934309BE
:100F5800E0914409E170E0934409EE0FA091430940
:100F6800EA0F0E2FE091D506EF5FE093D5060E94B9
:100F78001414FF93EF93E02FE05DAF91BF91EC93D2
:100F88000E944117239608951A930A93E091D50673
:100F9800E250E0934A06EAE4F6E0008113E0E091CB
:100FA800D5061E1730F4E12F0E9419140E0F1F5F8B
:100FB800F6CFE02F0E941E140E2F0A930E942614CB
:100FC800099119910895A091D506E0E0EA1710F467
:100FD8000E94D30FE0E0E093D606E093D506E093B5
:100FE8008D050895A0918D05A03021F427FE02C03B
:100FF80021FC01C00BC0A0914509A23029F4E0E012
:101008000E942C140E94FC05E89427F8A0918D05F5
:10101800A130D9F4E091D506A091D606AE1780F498
:10102800E0919B00E07259F0E091D606EF5FE09303
:10103800D6060E941414E081EA930E94890105C033
:10104800E0E0E0938D05E093D606A0918D05A230EF
:1010580011F40E94E7070895279781E0A0E0B0E027
:10106800E4EAF0E00E9445170E943717E09124084F
:10107800EB87E0912508EA87AB85AA3211F40C9436
:10108800B7080AE10E943014030FE02F0F5F0E9497
:1010980036140F5F0E943C144A3211F40C949F08D6
:1010A8000E9441140E944614E09126080E944F14A1
:1010B8000AE1202FE0917208E4502E1738F4E22F4D
:1010C8000E9456140E945B142F5FF4CF0E94601494
:1010D8000E946A14EF81E03069F5E09126080E94C9
:1010E8006E140AE10E943014E985E0934A06232F22
:1010F800E0E0E21758F4E02F0F5F0E945614103218
:1011080018F01A930E9482072150F2CFE02F0F5F48
:101118000E9436140F5F0E943C144A3259F00E9414
:101128006014EA930E942614E0914509E0938D0526
:10113800E1E0EE8317C007E10E947214232FE0E07C
:10114800E21758F4E02F0F5F0E9456140E947A1499
:10115800EC58F74F10832150F2CFEC85E0933E090D
:101168005093400918C007E10E947214EA85E09381
:101178004109232FE0E0E21758F4E02F0F5F0E94A7
:1011880056140E947A14E752F74F10832150F2CF79
:10119800EC85E0933F09EE81E03011F00C946F0983
:1011A800A0913E09E0E0EA1750F4A0913F09EA1740
:1011B80030F4E0914109A0914009EA1709F08BC089
:1011C800E0917408EB87E0917508EA870E94411462
:1011D800EDB7FEB7FA93EA931F9364D51F910E9467
:1011E80041140E944614E09176080E944F140E9410
:1011F800801423E0231738F40E948514E0810E94AC
:101208006A142F5FF7CF0E948A1425E0231738F459
:101218000E948F14E0810E946A142F5FF7CFE22F9B
:101228002F5F0E9494142F5F0E949A14EDB7FEB7A7
:10123800FA93EA931F9336D51F910E945B14EF81AE
:10124800E03011F00C946F09E09176080E946E145A
:10125800E0917408EB87E0917508EA870E944114D1
:10126800EDB7FEB7FA93EA931F931CD51F9110931D
:101278004A060E94801423E0231740F40E94851434
:1012880010811A930E9482072F5FF6CF0E948A145A
:1012980025E0231730F40E948F140E9484132F5FD7
:1012A800F8CFE22F2F5F0E9494142F5F0E949A14A8
:1012B800EDB7FEB7FA93EA931F93F4D41F911A93EC
:1012C8000E942614E0914509E0938D05E0E0E09343
:1012D8003E09E0933F090E943E172D960895E0913C
:1012E8003C07EF5FE0933C070E94A1140E94A614FC
:1012F800A0913C07A43618F0E0E0E0933C072DC02D
:10130800E091A307EF5FE093A3070E94AA140E944D
:10131800A614A091A307A43618F0E0E0E093A30771
:101328001CC0E0910A08EF5FE0930A080E94AF141E
:101338000E94A614A0910A08A43618F0E0E0E093F1
:101348000A080BC00E94B4140E94A614A091720847
:10135800A43618F0E0E0E0937208219608950E9400
:1013680039170E94B414DF01EC81EC93A091720844
:10137800A33618F0E0E0E0937208AC81A03210F0D8
:101388000C94DE0A0E94B414DF01E0E0EC93EDE077
:10139800F8E0FA93EA93E6E9F0E00E9401170E9468
:1013A800BA1411F00C94650AE0912408E03411F0A5
:1013B8000C94420AE0912508E43511F00C943B0A9C
:1013C800E09126080E94C214EF930E94C914AF91BD
:1013D800EA2311F40C943A0AE7E2F8E010810E943B
:1013E8002913EC56FD4F30810E942913EC56FD4F0E
:1013F8001083E02FF0E0FF93EF93E5E9F2E0AF917F
:10140800BF91FF93EF93E3E1F0E00E94C616AF911E
:10141800BF910E94CE1420E0EFE0E21718F1E02F10
:10142800F0E0FF93EF93E7E9F2E0AF91BF91FF930C
:10143800EF93E3E1F0E00E94C616AF91BF91AE0FC3
:10144800BF1FE22FF0E0EA0FFB1FFF93EF93E22F9D
:10145800EA5FF0E0E35FF74FE081AF91BF91EC9373
:101468002F5FDACF131711F0689427F806C0E091C0
:101478002508E23511F40E949E0522C0E091270854
:10148800E435F1F4E09128080E94C214EF930E9419
:10149800C914AF91EA23A1F0E02FF0E0FF93EF9396
:1014A800E5E9F2E0AF91BF91FF93EF93E3E1F0E05C
:1014B8000E94C616AF91BF910E94CE140E943008B8
:1014C80076C0EDE0F8E0FA93EA93EAE9F0E00E94EA
:1014D80001170E94D31481F4E0911308E053EF93AD
:1014E800E0911208E053AE2FEAE0EA9FE02DAF91B9
:1014F800EA0F2E2F622E5BC0EDE0F8E0FA93EA9334
:10150800ECE9F0E00E9401170E9490130E947816FF
:10151800E03039F5A0919302A030E4F0E091930215
:10152800F0E0FF93EF93EEE5F4E0AF91BF91FF9306
:10153800EF93E3E1F0E00E94C616AF91BF910E94DD
:101548003413E1E1EA93A09193020E94DB14EFEFD8
:10155800E0939302E1E0F0E0E0939002F0939102CF
:1015680026C0EDE0F8E0FA93EA93E0EAF0E00E94A2
:1015780001170E94D31471F4E1E0F0E0E0939002C7
:10158800F0939102A0919302A0301CF0EFEFE0934A
:1015980093020DC0EDE0F8E0FA93EA93EEE9F0E08B
:1015A8000E9401170E94BA1411F40E949E05E0E0FF
:1015B800E09372080E9440172596089523FE04C000
:1015C80024FC02C025FE01C037C0E0919002F091D2
:1015D8009102309781F5E0910A08A0910B08EA176B
:1015E800A9F05D9B12C0E0910B08EF5FE0930B0838
:1015F8000E94AF140E94E414A0910B08A43618F0BE
:10160800E0E0E0930B08689426F815C0E89423F806
:10161800E8ECF0E0E0939002F0939102A09193023D
:10162800EFEFEA1734F4E4EFF1E0E0939002F0937F
:101638009102E89426F84DC0E0919002F091910251
:10164800309711F00C946D0B20FE21C0E0913C07FF
:10165800A0913D07EA17A9F05D9B12C0E0913D07F4
:10166800EF5FE0933D070E94A1140E94E414A0914B
:101678003D07A43618F0E0E0E0933D07689424F8AD
:1016880005C0E89420F80E94E81424F822C022FE3D
:1016980020C0E091A307A091A407EA17A9F05D9BD9
:1016A80012C0E091A407EF5FE093A4070E94AA1478
:1016B8000E94E414A091A407A43618F0E0E0E09397
:1016C800A407689425F805C0E89422F80E94E81455
:1016D80025F808951A930A9310E0AA81A03010F013
:1016E800A83108F01CC000E0EFE0E017C0F0EA8184
:1016F800F0E0FF93EF93E7E9F2E0AF91BF91FF933A
:10170800EF93E3E1F0E00E94C616AF91BF910E940B
:10171800F0140E94391309F011E00F5FE5CFE12FB3
:1017280019810881239608952C970E943717EA8912
:10173800E09345090E94621300810E946D13108195
:101748000E946D13E081E0532E2F143529F42A935B
:101758000E946E0BE13009F006C1FE0136960E9428
:10176800F51430E0E8E0E31730F00E9401150E941C
:1017780073093F5FF7CF30E0EFE0E317B0F0E22FF7
:10178800F0E0FF93EF93E7E9F2E0AF91BF91FF93A9
:10179800EF93E3E1F0E00E94C616AF91BF910E947B
:1017A8000A150E9473093F5FE7CFECE2EA930E94B3
:1017B8007309309146063A93EDB7FEB7FA93EA9368
:1017C8004F93EDB7FEB7FA93EA935F934BD25F91CD
:1017D8004F910E941315E02FE05CEA930E94730971
:1017E800E1E0E0934306E3E0E98B0E946D13E081BA
:1017F800E88BA889A03228F0EA930E9473090E9416
:101808001915A889A03218F0A989A13408F001C0D7
:10181800ECCFA889A430B1F40E946D1330813A93BB
:10182800EDB7FEB7FA93EA934F93EDB7FEB7FA9385
:10183800EA935F9317D25F914F910E9413150E940C
:101848001D158FC0EAE2EA930E947309E0910C0823
:10185800EF5FE0930C08A0910C08E0E30E94BC162F
:10186800EF93EAE70E94C116AF91EA2B19F0E0E383
:10187800E0930C08E0910C08EA930E9473090E9417
:101888001D1530E0E8E0E31730F00E9401150E94D2
:1018980084093F5FF7CF30E0EFE0E317B0F0E22FC5
:1018A800F0E0FF93EF93E7E9F2E0AF91BF91FF9388
:1018B800EF93E3E1F0E00E94C616AF91BF910E945A
:1018C8000A150E9484093F5FE7CFECE2EA930E9481
:1018D8008409EAE2EA930E948409E0910C08EA93F9
:1018E8000E948409E2E3EA930E948409E4E5EA930A
:1018F8000E948409E22FE05DEA930E948409E0E0F7
:10190800E98B0E946D133081303228F03A930E949F
:1019180084090E941915303218F0A989A23308F0F9
:1019280001C0EFCF3430E9F40E946D1330813A934F
:10193800EDB7FEB7FA93EA934F93EDB7FEB7FA9374
:10194800EA935F938FD15F914F914A930E948409E4
:101958005A930E948409EDE0EA930E9484096894EE
:1019680022F8689420F80E943E176396089523FC95
:1019780041C0E1E4EA930E949509E4E5EA930E94F4
:101988009509EAE50E94211523F80E949201E09149
:101998009202F0E0FF93EF93EEE5F4E0AF91BF9190
:1019A800FF93EF93E3E1F0E00E94C616AF91BF9179
:1019B8000E943413EFEFE0939202E0939302A09118
:1019C8004509A23011F421FC01C014C00E94E707A8
:1019D8000E9499130E949E130E94D0130E948C1398
:1019E800E4E5EA930E948207EAE5EA930E94820707
:1019F8000E94DF13089523FC41C0A0914509A2303D
:101A080011F421FC01C03AC00E94E7070E94991313
:101A18000E949E130E94D013E9E4EA930E94820771
:101A2800EEE6EA930E948207E9E6EA930E948207BB
:101A3800E4E7EA930E948207E3E4EA930E948207BC
:101A4800AA810E942A15AA810E942E15AB810E94A4
:101A58002A15AB810E942E15E0E5EA930E948207C1
:101A6800A8810E942A15A8810E942E15A9810E948A
:101A78002A15A9810E942E150E94DF132496089525
:101A880064970A93A0919202A03014F40C94090E62
:101A980023FCBBC0E0E1EA93A09192020E94DB1410
:101AA800E0919202F0E0FF93EF93EEE5F4E0AF915E
:101AB800BF91FF93EF93E3E1F0E00E94C616AF9168
:101AC800BF910E94321528F00E9437150E94BB0C66
:101AD8009CC0FE0131960E94F51400E0E8E0E01792
:101AE80040F0E02FF0E0DE0111960E943C150F5FF8
:101AF800F5CF00E0EFE0E017B8F0E0919202F0E0F7
:101B0800FF93EF93EFE5F4E0AF91BF91FF93EF936D
:101B1800E3E1F0E00E94C616AF91BF910E94F01475
:101B28000E943C150F5FE6CFECE2EA930E9495090C
:101B3800E0E4EA930E949509E2E5EA930E94950998
:101B4800EAE2EA930E949509E0919202F0E0FF939D
:101B5800EF93EEE5F4E0AF91BF91FF93EF93E3E1EC
:101B6800F0E00E94C616AF91BF91AE0FBF1FEC9177
:101B7800E05DEA930E9495090E944215E05D0E948B
:101B8800211523F8E0919202F0E0FF93EF93EDE541
:101B9800F4E0AF91BF91FF93EF93E3E1F0E00E948F
:101BA800C616AF91BF910E943413E0919202F0E003
:101BB800FF93EF93EEE5F4E0AF91BF91FF93EF93BE
:101BC800E3E1F0E00E94C616AF91BF910E94321582
:101BD80098F4E0919202F0E0FF93EF93EEE5F4E0E1
:101BE800AF91BF91FF93EF93E3E1F0E00E94C61637
:101BF800AF91BF910E944B13E0919202E093930240
:101C08000E943715EFEFE0939202088165960895D8
:101C18000A93E981E150E983EF5FAA81BB81F0E093
:101C28000E94341309810030E4F0E02FAA81BB81BF
:101C3800F0E0EA0FFB1FFF93EF93AC81BD81EAE070
:101C4800F0E00E94FE16F096AF91BF91EC93AC8144
:101C5800BD81EAE0F0E00E94DC16EC83FD830150D0
:101C6800E2CF1DC00A930E9447150A3018F4E02FEE
:101C7800E05D02C0E02FE95CA981BA81EC93ED81B7
:101C8800E295EF70ED830E9447150A3018F4E02FB3
:101C9800E05D02C0E02FE95CAB81BC81EC93088178
:101CA800269608950A93AC81A03318F0E9E3EA1761
:101CB80008F403C0EC81E053EC83AC81A13418F044
:101CC800E6E4EA1708F404C0EC81E154E65FEC832B
:101CD800AB81A03318F0E9E3EA1708F403C0EB81FD
:101CE800E053EB83AB81A13418F0E6E4EA1708F47B
:101CF80004C0EB81E154E65FEB83EC81E295E07F81
:101D0800AB81EA0F0E2FA981BA810C930881259621
:101D180008950A93E0E0EABBEFEFEBBB0E944B1596
:101D2800E1E0E093650000000000000009B3E3E093
:101D3800E0936500E02F088122960895EFEFEABB53
:101D48000E944B15E881EBBBE2E0E09365000000E0
:101D580000000000E3E0E0936500229608950A93EE
:101D6800E0EEE5BBEAE0F0E0FA93EA930E94A11600
:101D7800E0E6E5BBE4EFF1E0FA93EA930E94A116EE
:101D8800EFE0EA930E948D0EE33311F00C940F0FED
:101D9800EEE0EA93E3E3EA930E94A20EEAE00E94EF
:101DA8005015E02FE07FE034B1F5689421F80E94E7
:101DB80055150E9464150E9468150E946D150E94B1
:101DC80072150E947615E4E00E947C150E946D153C
:101DD8000E948015E6E00E947C150E94A20EE7E0B2
:101DE8000E948415E9E00E948C150E947615ECE0AB
:101DF800EA930E947215EDE0EA93E8E0EA930E9404
:101E0800A20E0E945515E1E0EA930E94A20E0E94DC
:101E180090150E949615BAC30E94371721FC01C07D
:101E2800BAC00E949015ECE00E94501500FD01C058
:101E3800B2C00E949C15E7E0EA93E0EEEA930E94A4
:101E4800A20E11E0EAE0E11728F0E8E00E94501540
:101E58001F5FF8CF10E0E5E0E11758F00E949F15EA
:101E6800FF93EF930E94A415AF91BF91EC931F5F6E
:101E7800F2CF40E00E94A4155E2FE0E0E51708F4D9
:101E880088C00E94A4155E2F450FE8E00E945015F7
:101E9800043509F07EC0400FE8E00E945015023476
:101EA80009F077C0400F11E0511758F0E8E00E94A0
:101EB8005015A12FB0E0AA5BB64F0C93400F1F5FDF
:101EC800F3CF403009F065C010E0E5E0E11770F0AD
:101ED800E12FF0E0E35BF54FFF93EF930E949F152E
:101EE800E081AF91BF91EC931F5FEFCFE0E0E0930B
:101EF8004206535020E0E52FE150F0E0EA5BF64F50
:101F08001081103211F0103011F4515001C021E04D
:101F1800203019F4E2E0E51708F001C0ECCF11E039
:101F2800151798F4A0914206E0E6EA1760F00E94BF
:101F3800A815FF93EF93E12FF0E0EA5BF64FE081FD
:101F4800AF91BF91EC931F5FEBCFE0914206EF5F3B
:101F5800E09346063091460610E0E09142061E17CF
:101F680030F4E12F0E9477133E0F1F5FF6CFE32F67
:101F78000E941E143E2F0E945713E4E0EC930E9427
:101F8800A81530830E94B215E2E0EA930E94660425
:101F980002C00E94B2150E943E17269608950E941C
:101FA8003917DD24EEE0EA93E0E3EA930E94A20EFB
:101FB800E0E0EA93E1E8EA930E94A20EE1E0EA9306
:101FC8000E9472150E9490150E94B515ECE00E94BF
:101FD80050150E94BF1579F0E1E0DE2E0E9496159B
:101FE80085E08A95F1F70E94B5150E94BF1519F092
:101FF800E2E0DE2E72C0E3E00E945015E2E0EA93D0
:102008000A930E94A20E0E949C15E7E0EA93E0E47E
:102018000E94C3150E94C915E091D506E2501E2FF3
:10202800E8E0EA93E12FE65E0E94C31520E0E5E0D0
:10203800E21758F00E94CC15F0E0E35BF54FE08121
:10204800EA930E94A20E2F5FF2CFE8E00E947C156F
:102058000E94A20E0E94D015E8E00E947C150E9402
:10206800A20EE8E00E948415E8E00E948C150E9408
:10207800C915E8E0EA931A930E94A20E312FE8E00E
:102088000E947C150E94A20E3C5A0E94D0153E5B0D
:1020980023E0211768F40E94CC150E941914EA93D2
:1020A8000E94A20EE22F0E9419143E0F2F5FF1CF5B
:1020B800E32FE095EF5F3E2FE8E0EA933A930E9422
:1020C800A20E0E94C9150E94C9150E94C915E0E018
:1020D800EA93E0ECEA930E94A20E0E94401724962D
:1020E8000895ECE0E093590AE3E0E093530A089579
:1020F8000A93A6EAB0E0EC810E94D315AA81A13028
:1021080009F40058E02FE095EF70E06FE09362006B
:10211800E02FE095E695E695EC73E36CE3B9A6EA63
:10212800B0E0EB810E94D315A981A13009F40058D1
:10213800E02FE095E295E07FE07FEF60E8BBE02FDD
:10214800E095E07FE360E2BB0881259608950A9355
:10215800A091530AA13009F5E1E0EA93E2E10E9477
:10216800D8150E947C10A091540AA33080F0E2E0B8
:10217800E093530AECE0E093590A00E0063020F4BB
:102188000E94DE150F5FFACFE0E0E093630AE0916A
:10219800540AEF5FE093540A16C1A091530AA23083
:1021A80011F00C941F11E4E0E0938C05E091620AB1
:1021B800EF5FE093620AE091630AEF5FE093630ADE
:1021C800A091630AE2E3EA1708F4FFCFA091620A3C
:1021D800E1E0EA1718F4E0E0E093620AEBE0EA9342
:1021E800EA93E091620AE170EA93A091620AAF5F14
:1021F800EA2FE1700E94E5150E94F01500E0053015
:10220800C8F4E02F0E94F415EF3431F4E02FEF5FAB
:102218000E94F415EB3409F00BC0E0E0E093530A98
:10222800E2E0E0938C05ECE0E093590A0E94F9158E
:102238000F5FE5CFC8C0A091530AA33011F00C94EA
:10224800E7110E940116A091590AAA30F9F4EBE0AF
:102258000E94D815E0E0EA930E947C10E4E0E09345
:102268008C050E940716E4E5EA93A6D10E940B1696
:102278000E940F160E9413160E9417160E941D1620
:102288000E9421160E941D160E94F015A091590A5D
:10229800A93059F5EBE00E942C140E9427160E94E1
:1022A8000B160E942A160E9413160E940F160E94EF
:1022B8000F16A091550AEFE0EA1728F40E942A1693
:1022C8000E940F1610C00E940F16A091550AAA303E
:1022D80020F4E091550AE05D04C0E091550AEF5BF7
:1022E800EA50EA9369D10E94F015A091590AA830E2
:1022F80091F4EBE0EA93E3E0EA930E9427160E9448
:102308000B160E9407160E9413160E940F160E94B1
:102318000F160E94F015A091590AA730B9F4EBE006
:10232800EA930E946815E0E00E94E5150E940B16EA
:10233800E3E30E942E160E940F16E5E3EA933CD1D0
:102348000E942A160E940F160E94F015A091590AA1
:10235800A630C9F4EBE0EA93E5E0EA930E94271679
:102368000E940B16E8E30E942E16A0E0B0E00E943F
:102378001017E03011F4E0E301C0E2E3EA931CD166
:10238800E2E30E943216A091590AA53049F4EBE025
:10239800EA93E6E0EA930E942716EAE50E943216DD
:1023A800A091590AA43079F40E94F915E2E0E0936B
:1023B800530A00E0063020F40E94DE150F5FFACFC2
:1023C800E0E0E093630AE2C00A93A091530AE0E0D8
:1023D800EA1718F40E94AB10D9C0E0915A0AE150EC
:1023E800E0935A0AE03011F00C94CA12E2E0E0934C
:1023F8005A0A0E940116E0B1E095E295EF70E09369
:10240800550AE03019F4E0E1E093550A06B3E02FED
:10241800E170EF93E02FE695E670AF91EA0FEF9346
:10242800E02FEE0FEE0FE870AF91EA0FE093560A37
:10243800E095EF70E093560AA091590AE6E0EA1792
:1024480010F40E94440DA091590AA63031F4EAE034
:10245800EA930E9442150E943616A091590AA530A7
:1024680059F4A091550A0E943C16A091550AEAE039
:102478000E94FB160E943616A091590AA43039F41E
:102488000E941716EA930E9421160E943616A09100
:10249800590AA33071F4A72D0E943C16A72DEAE033
:1024A8000E94FB16EA93E0E0EA93E1E0EA930E94D7
:1024B8007C10A091590AA23021F5219781E0A0E073
:1024C800B0E0E4ECF0E00E944517A1E0B0E00E9423
:1024D8000C17E038A5E2FA0719F4E1E0E8830DC02B
:1024E800E030ABE4FA0719F4E2E0E88306C0E03034
:1024F800A6E9FA0711F4E3E0E883EEE00E9441164A
:102508002196A091590AA130A1F4219781E0A0E079
:10251800B0E0E6ECF0E00E944517A0E0B0E00E94D1
:102528001017E13011F4E1E0E883EFE00E94411672
:102538002196A091590AA03049F50E94F915E4E1C5
:10254800E093590AE091560AA091570AEA1731F424
:10255800E091550AA091580AEA17C1F0E091570A8C
:10256800EA93E091560AEA93E091580AEA93E091D7
:10257800550AEA930E94FF0CE091560AE093570A25
:10258800E091550AE093580A0E9475100991089540
:10259800E091610AEF5FE093610AE150F0E0E55AEB
:1025A800F54F0E94A614A091610AA63018F0E0E049
:1025B800E093610A219608955D9BFECFE881ECB90E
:1025C80021960895B981A881EC91EA930E944C164E
:1025D800EE2311F01196F8CFE894EC91ED3211F456
:1025E800689402C0EB3209F4119666277727EC91BC
:1025F800EA930E944416EE2381F0E62FF72F660F28
:10260800771F660F771F6E0F7F1F660F771FED917D
:10261800FF27E0536E0F7F1FEACFE62FF72F1EF438
:10262800E095F095319622960895AA93BA93EA9385
:10263800EFB7EA931A930A93089509911991E991CA
:10264800EFBFE991B991A9910895E02FF0E0A3E1D6
:10265800B0E00E94C6160895EC93E02FF0E00895CC
:10266800AE0FBF1FE0E0EC930895AE0FBF1FEC91D3
:10267800E0300895F0E0A3E1B0E00E94C6160895A6
:10268800E45AFB4FE081AE2FE0E0EA170895AE0F61
:10269800BF1FEC91EF5FEC930895E0914406EF5F64
:1026A800E09344060895E0914206EF5FE093420606
:1026B800E150F0E0EB54FA4FDF010895E0E0E093D9
:1026C8004306EF5FE0934306E150F0E0EB54FA4F26
:1026D8000895E0914306EF5FE0934306E150F0E090
:1026E800EB54FA4F0895F0E0EB54FA4FE081089567
:1026F800E7E4EA930C948207E3E5EA930C948207F3
:10270800E081EA930C948207EBE3EA930C94820746
:10271800E1E4EA930C948207FA93EA93E2E0EA93FD
:102728000895EA930E948207EFCFEEE0EA930E94B1
:102738007207E2CFE92DE05DEA930C948207E88105
:10274800EA930C94AA04A12FE0E30E94B716089517
:10275800A12FE9E30E94B2160895EE81EF5FEE83A0
:10276800E150F0E0DE0117960895AE0FBF1FE02F8D
:10277800F0E0AE0FBF1FEC91EA930C948207FA9336
:10278800EA93E0E1F0E0FA93EA930895E45AFB4F04
:10279800DF01EAEFEC930895EAE2EA930E948207E8
:1027A800EAE2BFCFEA930E948207E9810895E05DDB
:1027B800EA930C9482070E94C807E2E0E0938D0533
:1027C8000C94E7070E94C807E1E0E0938D0508959F
:1027D800E0914206E150A09143060895E150F0E0EF
:1027E800E35FF74F0895E981EA93E981EA93089551
:1027F800E093D506EF5FE093D506E150F0E0E85BA3
:10280800F94FDF010895EC93E091D506EF5F089545
:10281800E093D506E150F0E0E85BF94FDF01089559
:10282800E150F0E0E85BF94F0895F0E0E85BF94F1C
:10283800E0810895A0E0B1E0F0E00E940517EA1BEE
:10284800FB0B08950E948207EDE0EA930C9482073F
:10285800EA93E2E0EA930895E0917208E01BE450FD
:102868003E2F0895F0E0E35FF74F4081E02F089591
:10287800F0E0E35FF74F50810895EB85EA93EB852D
:10288800EA930895FE013B96FA93EA930E94560E46
:10289800E985EF830895E0541E2FE12FAF81EA0FF9
:1028A800EF830895F0E0E35FF74F10810895E12F7B
:1028B800AF81EA0FEF8308954A935A93FE013A963F
:1028C800FA93EA930E94560EE8850895AF81EA0FBD
:1028D800EF830895E054EA930C947207E09172082C
:1028E800E01BE2503E2FE0E0EC870895EC85EF5FB7
:1028F800EC87E150F0E00895E0913E09E2503E2F68
:102908000895E22FF0E0EC58F74F0895E0913F0961
:10291800E2503E2F0895E22FF0E0E752F74F089576
:10292800F0E0E752F74F4081E22F0895F0E0E752D8
:10293800F74F50814A935A930895E150F0E0E952D5
:10294800F94F0895DF01E881EC930895E150F0E034
:10295800E25CF84F0895E150F0E0EB55F84F089528
:10296800E0917208EF5FE093720838CFFA93EA9328
:10297800E6E0EA930E947816E0300895E0530E2FBF
:10298800A02FE0E00E94B7160895A02FE8E10E946A
:10299800BC160895AE0FBF1FE4E0EC930895FA93B8
:1029A800EA93E5E0EA930E947816E0300895EAE0B9
:1029B8000E94EF16EA93E0E0EA93EA930C947C1005
:1029C800E081EA930C94E012E8ECF0E0E0939002E6
:1029D800F0939102E8940895AE0FBF1FE02FF0E046
:1029E8000895FA93EA93E8E9F0E00E940117FA9350
:1029F800EA93E9E0EA930C948D16E32FF0E0DE0108
:102A08001696AE0FBF1FEC91EA930895AE0FBF1F45
:102A1800E32FF0E0AE0FBF1FEC91EA9308954A93BD
:102A28000E9473095A930C947309E989EF5FE98B43
:102A38000895EDE0EA930C947309EA930E949509CE
:102A4800EDE0EA930E94950968940895EAE00E94EF
:102A5800CE16ADCEEAE00E94FB16A9CEAE0FBF1F80
:102A6800AC91A6300895E0919202EA930C940A067C
:102A7800AE0FBF1FEC91EA930C949509A92DEAE0DB
:102A88000E94FB160895ED81EF700E2F0895E981DD
:102A9800EF71E066E5BB0895EA930E948D0E0E2F54
:102AA8000895EEE0EA93E0E3EA930E94A20EE4E0E0
:102AB800EA93E0E0EA930E94A20EE5E0EA93089523
:102AC800E0E8EA930C94A20EE4E0EA93E0E0EA93EB
:102AD80008950E94A20EE5E0EA930895E0E0EA93E3
:102AE8000C94A20EEEE0EA93E1E3EA930C94A20EB2
:102AF800EA93E4E5EA930895E2E4EA930C94A20EDB
:102B0800EA93E3E5EA930E94A20EE8E0EA93E6CFAF
:102B1800EA939A920C94A20EEEE0EA93E2E3EA9327
:102B28000C94A20EE0E0EA93E0E4EA930C94A20E7F
:102B3800E6E0EA93D3CFE12FF0E0E95BF54F0895A3
:102B4800E8E0EA930C948D0EE0914206EF5FE09383
:102B58004206E150F0E0EB54FA4F0895E0E0EA93C2
:102B6800AFCFE0E0EA93E1E2EA930E94A20E85E0AB
:102B78008A95F1F70895E02FE470E4300895EA9318
:102B88000E94A20EE8E0EA93A9CFE8E0EA93A6CF74
:102B9800E8E0EA93E22F0895E8E0EA93ADCFF0E0A9
:102BA800EA0FFB1F04910895EA93E1E0EA93E0E05D
:102BB800EA930895A02FB0E0A55AB54FE0E0EC9352
:102BC8000895EA930E947C10E1E4EA930E94E012DF
:102BD800E4E5EA930C94E012EDE0EA930C94E01239
:102BE800F0E0E55AF54FE0810895EAE0EA93EA93C8
:102BF800E0E0EA93EA930C947C10E091590AE150E2
:102C0800E093590A0895E1E4EA930C94E012E3E5AD
:102C1800EA930C94E012E0E3EA930C94E012EDE3FB
:102C2800EA930C94E012A091560AEAE00E94CE16AC
:102C38000895E05DEA930C94E012A091560AEAE048
:102C48000E94FB160895E0E0EA93BBCFE1E3EA9324
:102C58000C94E012EA930E94E012E1CFEA930E94FA
:102C6800E012BACFEA93E0E0EA93EA930C947C107E
:102C7800EAE00E94CE16EA930895EA93E981F2CF3A
:102C8800E1E0F991F03310F0FA3308F0EE270895F7
:102C9800E1E0F991F03229F0F93010F0FE3008F057
:102CA800EE2708956627772789919991E991F991F7
:102CB800A991B991009629F001976D9171916717C3
:102CC800C9F3671BE62F089599818881009641F022
:102CD800BD81AC81FB81EA8161916D930197E1F738
:102CE800FD81EC8126960895002411246991E991CB
:102CF800F991A991B991662349F06A951D900590BB
:102D0800011421F40020B9F7EE2702C01018E12DB4
:102D180008956991E991F991A991B991CD01662335
:102D280051F06A9505900D920020C9F7662319F0B5
:102D38006A950D92FBCFFC010895E991F9913096BF
:102D480039F080EA9FE00197F1F7A8953197C9F724
:102D58000895EA17E1E009F0EE270895EA17E1E09F
:102D680008F4EE270895AE17E1E008F4EE27089579
:102D7800AE17E1E008F0EE270895EA17E1E008F061
:102D8800EE270895FA9FF02DEB9FF00DEA9FE02DB6
:102D9800F10D0895002498E0AA0F001C0E1A10F4F3
:102DA8000E0E01C0A1609A95B9F7EA2FA02D0895DB
:102DB8000024112490E1AA0FBB1F001C111C0E1A3D
:102DC8001F0A18F40E0E1F1E01C0A1609A9599F7EC
:102DD800FD01D0010895E894A7FF02C0A195689469
:102DE800E7FDE195D7DFEA2F0EF4E1950895D2DFEC
:102DF800EA2F0895DDDFFD0108950590F491E02D97
:102E080008951B2EBF2FF12D1A2EAE2FE12D0895F8
:102E1800119602D0FE2F1197E199FECFFF93FFB7CD
:102E2800F894AEBBBFBBE09AEDB3FFBFFF91089526
:102E380007D01196EF93EF2F03D0EF9111970895D4
:102E4800E199FECF9FB7F894AEBBBFBBE09A8DB3B4
:102E5800E81719F0EDBBE29AE19A9FBF08950024A4
:102E68000A160B0608955A934A933A932A931A938B
:102E78000A9308955D814C813B812A8119810881DB
:102E88000895AC0FBD1F05900D928A95E1F708953E
:00000001FF
